:1062F8009005A27427F0A37410F09005A274FFF51E
:0F630800F01245EFFED3E5F09400EE940050EB59
:106317007D017F04125FAD12680F1263761269EB7D
:10632700126A521268F212661012694612695F0207
:026337006A32C8
:105FAD00AE8475840F758A83E4F59775840FF58932
:105FBD00F58475B73075840F4389018D8D758F010B
:105FCD008F8EFDFC0DBD00010CE4B505F7ECB401A1
:105FDD00F3438902E58920E4120DEDAA0470010C4A
:105FED0014D39400EA6480948140E9759702AF065A
:025FFD008F848F
:015FFF00227F
:10680F00AF8475840F75E10343E20443E3C075A4BD
:10681F000F7580F075A51775AD17E4F5A675A7F080
:02682F008F8454
:016831002244
:0D6A5200AF84E4F58475D48475D1038F847E
:016A5F002214
:1069EB00AF84E4F584759D0443F808759A40D2F89A
:0269FB008F8487
:0169FD002277
:10694600AF84758401E4F5C975CA3C75CB5D75CD18
:086956006E75CCACF5C88F840E
:01695E002216
:10695F00AF84758402E4F5C975CA1975CBFF75CD7F
:08696F00FF75CC19F5C88F84F7
:0169770022FD
:106610009005A4E584F0E4F584F5BA75BC9875E8B6
:10662000C0758402F5BA75BC9043BC0175E8C075AD
:0E663000C4AF75C6FF1265B09005A4E0F584F6
:01663E002239
:106A320043E701D2A8D28A43E70443F704D2AF2244
:065F5400C10D4107B6007B
:10657C00AE8475840F75A40F7580F075A7F0E4FDDB
:10658C00FC0DBD00010CBC4EF8BD20F5E58030E6DD
:10659C0004E4FF800CE5B0540F70047F018002E42A
:0365AC00FF8E84DB
:0165AF0022C9
:1066CC009008C7E0FEA3E0FF9008C3E0FCA3E0FD48
:1066DC00B50719ECB506159008CCE0FEA3E0FFED6C
:0E66EC00B50709ECB5060520C502D322C3226E
:102AB10075FFDE75FFADE4F5E6F5E79007B83094F4
:102AC100057444F080037445F01262F8126A10E450
:102AD1009006C4F09007B07407F0E49007B4F0904A
:102AE10006C3F09004B6F09006BF12474B000000F9
:102AF10000E49007B1F004A3F0E4900909F0126832
:102B01009412669D9007B3E0FF126A21126A601267
:102B11006463126AA6125A20126A7CE49006BDF020
:102B21009007B9F075840143C80475840243C80451
:102B3100F5849007BBF09007B904F075840F126516
:102B4100E0EF7003022CDA900902E0FFB40B02D22D
:102B51000DEF643170449007B8E0FF900903E06F16
:102B610070381266CC50FB9007B8E0FF1269D6129C
:102B710066CC50FB900904E0FFA3E0FDA3E0FBA3BA
:102B8100E09005A5F01252F51266CC50FB9007B803
:102B9100E0FF1269C11266CC50FB900902E0643279
:102BA10070449007B8E0FF900903E06F7038126637
:102BB100CC50FB9007B8E0FF1269D61266CC50FBEF
:102BC100900904E0FFA3E0FDA3E0FBA3E09005A5CD
:102BD100F012189A1266CC50FB9007B8E0FF126908
:102BE100C11266CC50FB900902E0642D704390073E
:102BF100B8E0FF900903E06F70371266CC50FB908C
:102C010007B8E0FF1269D61266CC50FB900904E0C8
:102C1100FFA3E0FDA3E0FB1258441266CC50FB90E9
:102C210007B8E0FF1269C11266CC50FBE4900903BA
:102C3100F0900902E0642E703E9007B8E0FF900921
:102C410003E06F70321266CC50FB9007B8E0FF12C0
:102C510069D61266CC50FB900904E0FFA3E0FDA306
:102C6100E0FB1257381266CC50FB9007B8E0FF1218
:102C710069C11266CC50FB900902E0FFB4140C90BC
:102C810006C374FFF09007B97401F0EFB4150AE4BC
:102C91009006C3F09007B904F09006C3E0603A9043
:102CA1000902E0146021047030900903E0FFC3942D
:102CB1001E5026900909EFF012669D9006BD740121
:102CC100F09007B9F08012900903E0FFC3941E5001
:102CD10008900909EFF0126AAC12690FEF70030254
:102CE100322A12621FEFB414004003023221902CE9
:102CF100F6F8282873022D32022D5B022D7A022D5F
:102D010064022D8D022DA9022F22022F3C022F5683
:102D1100022FC60230350230A4022E45022EB40223
:102D210031120231810231F9023201022D4E023299
:102D31001F300D099006C3E0F4F0022E3FE4900924
:102D410009F0126AACE49007BBF0022E3F9007B87D
:102D5100E0FF7D0A1268740232219007B4E0F4F0BA
:102D6100022E3F9007AFE004F0A3E0FF9007AFE031
:102D7100D39F4031E4F00231ED9007AEE0F4F0E48E
:102D81009007B1F09007B904F00232219006C4E037
:102D910004F0E0FFB40304E4F0800AEFB4FF06900E
:102DA10006C47402F00231ED9007AFE0FF75F01D2B
:102DB100A424C9F582E43406F583C083C082900659
:102DC100C4E0FED082D08375F00912477CE004F0A4
:102DD100EF75F01DA424C9F582E43406F58375F07E
:102DE10009EE12477CE0FFB408279007AFE075F0C9
:102DF1001DA424C9F582E43406F583C083C0829002
:102E010006C4E0D082D08375F00912477CE4F080DB
:102E11002AEFB4FF269007AFE075F01DA424C9F591
:102E210082E43406F583C083C0829006C4E0D08278
:102E3100D08375F00912477C7407F0121A069007C7
:102E4100B902321A9007AFE0FF75F01DA424C5F551
:102E510082E43406F583C083C0829006C4E0FED0CC
:102E610082D08375F00912477CE004F0EF75F01D04
:102E7100A424C5F582E43406F58375F009EE124702
:102E81007CE0D3945540269007AFE075F01DA42453
:102E9100C5F582E43406F583C083C0829006C4E0A0
:102EA100D082D08375F00912477C7455F0121A064E
:102EB1000231ED9007AFE0FF75F01DA424C5F58246
:102EC100E43406F583C083C0829006C4E0FED0825C
:102ED100D08375F00912477CE014F0EF75F01DA462
:102EE10024C5F582E43406F58375F009EE12477CBA
:102EF100E0D3945540259007AFE075F01DA424C59B
:102F0100F582E43406F583C083C0829006C4E0D024
:102F110082D08375F00912477CE4F0121A0602315F
:102F2100ED90083CA3E0FAA3E0F5828A837F0112C9
:102F310047B2121A069006BD02321A90083CA3E06D
:102F4100FAA3E0F5828A837FFF1247B2121A069034
:102F510006BD02321A9007AFE0FF75F01DA424C62A
:102F6100F582E43406F583C083C0829006C4E0FE96
:102F7100D082D08375F00912477CE02402F0EF750E
:102F8100F01DA424C6F582E43406F58375F009EE3C
:102F910012477CE0D3946340269007AFE075F01DA3
:102FA100A424C6F582E43406F583C083C08290066A
:102FB100C4E0D082D08375F00912477C7463F012AB
:102FC1001A060231ED9007AFE0FF75F01DA424C68B
:102FD100F582E43406F583C083C0829006C4E0FE26
:102FE100D082D08375F00912477CE024FEF0EF75A2
:102FF100F01DA424C6F582E43406F58375F009EECC
:1030010012477CE0D3946340259007AFE075F01D33
:10301100A424C6F582E43406F583C083C0829006F9
:10302100C4E0D082D08375F00912477CE4F0121A13
:10303100060231ED9007AFE0FF75F01DA424C7F53E
:1030410082E43406F583C083C0829006C4E0FED0DA
:1030510082D08375F00912477CE004F0EF75F01D12
:10306100A424C7F582E43406F58375F009EE12470E
:103071007CE0D3946340269007AFE075F01DA42453
:10308100C7F582E43406F583C083C0829006C4E0AC
:10309100D082D08375F00912477C7463F0121A064E
:1030A1000231ED9007AFE0FF75F01DA424C7F58252
:1030B100E43406F583C083C0829006C4E0FED0826A
:1030C100D08375F00912477CE014F0EF75F01DA470
:1030D10024C7F582E43406F58375F009EE12477CC6
:1030E100E0D3946340259007AFE075F01DA424C799
:1030F100F582E43406F583C083C0829006C4E0D033
:1031010082D08375F00912477CE4F0121A0602316D
:10311100ED9007AFE0FF75F01DA424C8F582E434FB
:1031210006F583C083C0829006C4E0FED082D083BE
:1031310075F00912477CE02402F0EF75F01DA4241C
:10314100C8F582E43406F58375F009EE12477CE098
:10315100D3946340269007AFE075F01DA424C8F511
:1031610082E43406F583C083C0829006C4E0D08235
:10317100D08375F00912477C7463F0121A06806CD3
:103181009007AFE0FF75F01DA424C8F582E4340672
:10319100F583C083C0829006C4E0FED082D08375DF
:1031A100F00912477CE024FEF0EF75F01DA424C85D
:1031B100F582E43406F58375F009EE12477CE0D31D
:1031C100946340259007AFE075F01DA424C8F582F3
:1031D100E43406F583C083C0829006C4E0D082D077
:1031E1008375F00912477CE4F0121A069006BD744B
:1031F10001F09007B9F080281268549006BD80193B
:103201009007B6E0F4F07005121A1B800990800057
:10321100E4939007B3F09006BD7401F0800280FE44
:1032210012690FEF6003022CE39007B9E060081206
:10323100374DE49007B9F09006BDE07003022B3CD6
:0B324100126A7CE49006BDF0022B3CFA
:1068F2007F809007BCE4F0A3DFFC7B017A0779BCC0
:0C6902008B0A8A0B890C8A088909D2B420
:01690E002266
:10690F00E50A850B83850C826401700AE5096582AF
:0D691F007004E50865837002FF227F0122ED
:10621F00E50A850B83850C826401700AE5096582A6
:10622F007004E50865837003FF802FAB0A050CE54A
:10623F000CAA0B7002050B14F912453BFF74019069
:10624F00083C6B700AE50C65827004E50B65837082
:0A625F0009750A01750B07750CBCE8
:016269002212
:031A0300025E94EC
:105E9400C0E0C083C082C0D075D000C004C005C0BB
:035EA40006C0072E
:105EA700AF8475840FE5B0540FFEE580548013135B
:105EB70013541F4EFE0509E509AC087002050814C6
:105EC700F5828C83EEF0C3E509943CE5089408401D
:105ED700067508077509BCC2B43086FDD2B48F8435
:105EE700D007D006D005D004D0D0D082D083D0E060
:015EF7003278
:105F5A004308964020104808994010040140100454
:105F6A000148088E80200802802008024808B102F1
:105F7A00020202010101014808A102020202010112
:105F8A0001014808B900020408060A0C0E4808A9CB
:085F9A000002040601030507E3
:10374D009005A3E5E7F0121A0C9007AEE0FD6007B7
:10375D00900886E04480F0900886E0FF9006C4E073
:10376D00FE2496F582E43408F583E0FCEF4C9008D6
:10377D0086F0ED700302380A9007ADE06025C39026
:10378D0004B4E09401501C9008B1E02486F582E465
:10379D003408F583C083C082E0FF900899E0FDEF07
:1037AD004D8055900416E09007B16023E024B1F5EB
:1037BD0082E43408F583E02486F582E43408F58349
:1037CD00C083C082E0FF900899E0FDEF4D8029E0B5
:1037DD00FF24B1F582E43408F583E02486F582E414
:1037ED003408F583C083C082E0FD74992FF582E41F
:1037FD003408F583E0FFED4FD082D083F09007AF12
:10380D00E0FF24A1F582E43408F583E02486F582F7
:10381D00E43408F583C083C082E0FD748E2FF582F9
:10382D00E43408F583E0FFED4FD082D083F09008AB
:10383D0086E0FF9007AFE0FD75F01DA424C9F58269
:10384D00E43406F58375F009EE12477CE025E0FEC1
:10385D00EF4E900886F090088CE0FF9007B4E0548E
:10386D0040FEEF4E90088CF0300D07E0FF9006C340
:10387D00800890088CE0FF9007BBE05480FEEF4E6F
:10388D0090088CF09007AEE0FF60079007B1E0FE66
:10389D008002AE05EE75F01DA424C9F582E4340650
:1038AD00F583E024A9F582E43408F583E0C43333CD
:1038BD0054C090088DF0E0FEEF60079007B1E0FF77
:1038CD0080059007AFE0FFEF75F01DA424D2F582BF
:1038DD00E43406F583E024A9F582E43408F583E0A9
:1038ED0033333354F84E90088DF0E0FF9007AEE07F
:1038FD0060079007B1E0FE80059007AFE0FEEE7522
:10390D00F01DA424DBF582E43406F583E024A9F54B
:10391D0082E43408F583E04F90088DF09007AFE016
:10392D0075F01DA424C7F582E43406F583C083C069
:10393D00829006C4E0D082D08375F00912477CE0F6
:10394D00FFC39450400890088B740FF0802DEFC387
:10395D00943C400890088B7427F0801FEFC3942887
:10396D00400890088B7433F08011EFC394149008C5
:10397D008B40057439F08003743CF09007AFE0750F
:10398D00F01DA424C6F582E43406F583C083C082FD
:10399D009006C4E0D082D08375F00912477CE0FD1B
:1039AD00C39450400990088CE0440FF08054EDC34F
:1039BD00943C400990088CE04427F080459007AF77
:1039CD00E075F01DA424C6F582E43406F583C083AA
:1039DD00C0829006C4E0D082D08375F00912477C76
:1039ED00E0FDC39428400990088CE04433F0801228
:1039FD00EDC3941490088CE040054439F0800344E5
:103A0D003CF09007AFE075F01DA424C8F582E434B6
:103A1D0006F583C083C0829006C4E0D082D0837542
:103A2D00F00912477CE0FDC394504009900889E0ED
:103A3D00440FF08054EDC3943C4009900889E04454
:103A4D0027F080459007AFE075F01DA424C8F582DE
:103A5D00E43406F583C083C0829006C4E0D082D0E2
:103A6D008375F00912477CE0FDC394284009900846
:103A7D0089E04433F08012EDC39414900889E0403E
:103A8D00054439F08003443CF09007AFE075F01D1C
:103A9D00A424C5F582E43406F583C083C082900664
:103AAD00C4E0D082D08375F00912477CE0FDC39449
:103ABD0048400A90088AE0443FF0023B61EDC39410
:103ACD003C400A90088AE0449FF0023B619007AFAA
:103ADD00E075F01DA424C5F582E43406F583C0839A
:103AED00C0829006C4E0D082D08375F00912477C65
:103AFD00E0FDC39430400990088AE044CFF0805433
:103B0D00EDC39424400990088AE044E7F080459085
:103B1D0007AFE075F01DA424C5F582E43406F583E6
:103B2D00C083C0829006C4E0D082D08375F00912A4
:103B3D00477CE0FDC39418400990088AE044F3F0F7
:103B4D008012EDC3940C90088AE0400544F9F08092
:103B5D000344FCF053E7FEC291E4FFE4FE74862FAC
:103B6D00F582E43408F583E0FDA806088002C3134E
:103B7D00D8FC139292E49005A2F09005A2E004F017
:103B8D00E0B414F6D290E49005A2F09005A2E00402
:103B9D00F0E0B414F6C2900EEEB408C10FEFB40805
:103BAD00BAD291E49005A2F09005A2E004F0E0B441
:103BBD0014F6C2919007AEE060079007B1E0FF8068
:103BCD00059007AFE0FFEF75F01DA424C9F582E461
:103BDD003406F583E030E104D2928002C292900562
:043BED00A3E0F5E775
:013BF10022B1
:0A1A0C007F08900886E4F0A3DFFCD9
:011A160022AD
:10324C002E3031002E3032002E3033002E30340030
:10325C002E3035002E3036002E3037002E30380010
:10326C002E3039002E3130002E3132002E31340008
:10327C002E3136002E3138002E3230002E323500F1
:10328C002E3330002E3335002E3430002E343500E2
:10329C002E3530002E3630002E3730002E383000D0
:1032AC002E393000312E3000312E3200312E3400C8
:1032BC00312E3600312E3800322E3000322E3500B1
:1032CC00332E3000332E3500342E3000342E3500A2
:1032DC00352E3000362E3000372E3000382E300090
:1032EC00392E300031302E004672656500537573EF
:1032FC007400456E626C0050756C730053746F7083
:10330C00004379636C0020203331002020333300DC
:10331C002020333500202033370020203339002083
:10332C00203431002020343400202034360020207A
:10333C00343900202035320020203535002020354E
:10334C003800202036320020203635002020363937
:10335C00002020373300202037380020203832005E
:10336C002020383700202039330020203938002025
:10337C0031303400203131300020313137002031F0
:10338C0032330020313331002031333900203134D5
:10339C0037002031353600203136350020313735B5
:1033AC0000203138350020313936002032303800D9
:1033BC0020323230002032333300203234370020B8
:1033CC003236320020323737002032393400203385
:1033DC00313100203333300020333439002033377F
:1033EC003000203339320020343135002034343071
:1033FC000020343636002034393400203532330086
:10340C002035353400203538370020363232002054
:10341C003635390020363939002037343000203722
:10342C00383400203833310020383830002039331C
:10343C0032002039383800313035300031313130FC
:10344C00003131373000313234300031333230001A
:10345C0031343030003134383000313537300031D0
:10346C0036363000313736300031383630003139AD
:10347C0038300032303930003232323000323335AD
:10348C003000323439300032363430003237393093
:10349C0000323936300033313430003333323000BF
:1034AC003335323000333733300033393530003474
:1034BC00313930002531733A253264202531733A85
:1034CC00253264202531733A257300610041006276
:1034DC00004200660046002531733A2532642043D1
:1034EC006E74726C20566C746765006D004D00250F
:1034FC0031733A2532642025347320543A253373C2
:10350C0000436F6E74726173742025316420202027
:10351C0020202000202020202020202020202020BF
:10352C002020202000204142434445464748494A38
:10353C004B4C4D4E4F505152535455565758595A57
:10354C006162636465666768696A6B6C6D6E6F70E7
:10355C007172737475767778797A30313233343599
:10356C00363738397E21402324255E262A28292DFA
:10357C002B3D7CFF324CFF3250FF3254FF3258FF50
:10358C00325CFF3260FF3264FF3268FF326CFF3214
:10359C0070FF3274FF3278FF327CFF3280FF32844E
:1035AC00FF3288FF328CFF3290FF3294FF3298FF4B
:1035BC00329CFF32A0FF32A4FF32A8FF32ACFF32A4
:1035CC00B0FF32B4FF32B8FF32BCFF32C0FF32C49E
:1035DC00FF32C8FF32CCFF32D0FF32D4FF32D8FFDB
:1035EC0032DCFF32E0FF32E4FF32E8FF32ECFF3234
:1035FC00F0FF32F4FF32F9FF32FEFF3303FF3308E2
:10360C00FF330DFF3312FF3317FF331CFF3321FF42
:10361C003326FF332BFF3330FF3335FF333AFF3381
:10362C003FFF3344FF3349FF334EFF3353FF3358CF
:10363C00FF335DFF3362FF3367FF336CFF3371FF82
:10364C003376FF337BFF3380FF3385FF338AFF33C1
:10365C008FFF3394FF3399FF339EFF33A3FF33A8BF
:10366C00FF33ADFF33B2FF33B7FF33BCFF33C1FFC2
:10367C0033C6FF33CBFF33D0FF33D5FF33DAFF3301
:10368C00DFFF33E4FF33E9FF33EEFF33F3FF33F8AF
:10369C00FF33FDFF3402FF3407FF340CFF3411FFFE
:1036AC003416FF341BFF3420FF3425FF342AFF343B
:1036BC002FFF3434FF3439FF343EFF3443FF34489A
:1036CC00FF344DFF3452FF3457FF345CFF3461FF3D
:1036DC003466FF346BFF3470FF3475FF347AFF347B
:1036EC007FFF3484FF3489FF348EFF3493FF34988A
:1036FC00FF349DFF34A2FF34A7FF34ACFF34B1FF7D
:10370C0034B6FF34BB0105FF54A5010EFF5CC100AC
:10371C0000FF60000005FF604E000AFF609C010086
:10372C00FF60EA0105FF54A50000FF60000005FFE3
:10373C00604E000AFF609C0100FF60EA0009FF6612
:01374C003F3D
:0E6A6000E4900863F0900862F0900861F02264
:066AA000E4900842F02220
:105C2C009005A2EEF0A3EFF0AF051DEF7003025C40
:105C3C00C09005A2E0FEA3E0F5828E83A3A3E493BB
:105C4C00FB740193FA740293F9900842E0FF75F02B
:105C5C0005A42445F582E43408F583EBF0A3EAF0BF
:105C6C00A3E9F09005A2E0FAA3E0FBF5828A83E4B5
:105C7C0093FEEF75F005A42443F582E43408F58314
:105C8C00EEF08B828A83740193FF900842E075F0EA
:105C9C0005A42444F582E43408F583EFF09008421F
:105CAC00E004F09005A3E02405F09005A2E0340098
:055CBC00F0025C34223F
:105D4400900842E0FF607490083FE0FBA3E0FAA3F0
:105D5400E0F912453BC39F4004E412457690083FA6
:105D6400E0FBA3E0FAA3E0F912453BFE75F005A4BD
:105D74002443F582E43408F583E0FFEE75F005A4CE
:105D84002444F582E43408F583E0FD1269AA9008FE
:105D94003FE0FBA3E0FAA3E0F912453B75F005A44C
:105DA4002445F582E43408F583E0F9A3E0FAA3E09E
:0C5DB40090083CC9F0A3EAF0A3E9F0223B
:1068540090083FE0FBA3E0FAA3E0F9740112455469
:1068640012453BFF900842E0B50704E41245762246
:10663F00D3EF6480948040119007B3E004F0E0D36F
:10664F00940740137407F0800E9007B3E014F0E046
:0F665F00D394074002E4F09007B3E0FF026A21F2
:1054A5009007ADE060030255BAD3EF648094804065
:1054B5006C9007AFE0FD75F01DA424E1F582E4349E
:1054C50006F583E004F0ED75F01DA424E1F582E412
:1054D5003406F583E0FDD3940540219007AFE075D0
:1054E500F01DA424E1F582E43406F5837405F090FB
:1054F50007AD7401F09007B07407F022ED64046005
:10550500759007AFE075F01DA424E1F582E434063B
:10551500F583E06405600302561D0255E29007AF6E
:10552500E0FD75F01DA424E1F582E43406F583E081
:1055350014F0ED75F01DA424E1F582E43406F5833D
:10554500E0FDD3940540149007AFE075F01DA42449
:10555500E1F582E43406F583E4F022ED6404601697
:105565009007AFE075F01DA424E1F582E43406F55B
:1055750083E0FDB405028065ED6403600302561DFA
:105585009007B07407F09007AFE004FEEEC39408EF
:10559500400302561DEE75F01DA424E1F582E434A6
:1055A50006F583E0FD64046004EDB405059007B0DD
:1055B500EEF00E80D7D3EF64809480505BE49007C3
:1055C500ADF09007AFE075F01DA424E1F582E43459
:1055D50006F583E0FF64046004EFB405099007AFA6
:1055E500E09007B0F0229007B07407F09007AFE0A5
:1055F50004FEEEC394085020EE75F01DA424E1F5D9
:1056050082E43406F583E0FF64046004EFB4050525
:085615009007B0EEF00E80DA00
:01561D00226A
:105CC100D3EF64809480403E9007AFE0FF75F01DF4
:105CD100A424E0F582E43406F583E004F0EF75F0E6
:105CE1001DA424E0F582E43406F583E0C394294041
:105CF100519007AFE075F01DA424E0F582E434066D
:105D0100F5837429F0229007AFE0FF75F01DA424FC
:105D1100E0F582E43406F583E014F0EF75F01DA49C
:105D210024E0F582E43406F583E0C394294013901E
:105D310007AFE075F01DA424E0F582E43406F58395
:035D4100E4F02269
:10600000D3EF648094809007AFE075F01D4020A42A
:1060100024CAF582E43406F583C083C0829006C4A6
:10602000E0D082D08375F00912477C7401F022A47D
:1060300024CAF582E43406F583C083C0829006C486
:0E604000E0D082D08375F00912477CE4F02294
:10604E00D3EF648094809007AFE075F01D4020A4DC
:10605E0024CBF582E43406F583C083C0829006C457
:10606E00E0D082D08375F00912477C7401F022A42F
:10607E0024CBF582E43406F583C083C0829006C437
:0E608E00E0D082D08375F00912477CE4F02246
:10609C00D3EF648094809007AFE075F01D4020A48E
:1060AC0024CCF582E43406F583C083C0829006C408
:1060BC00E0D082D08375F00912477C7401F022A4E1
:1060CC0024CCF582E43406F583C083C0829006C4E8
:0E60DC00E0D082D08375F00912477CE4F022F8
:1060EA00D3EF648094809007AFE075F01D4020A440
:1060FA0024CDF582E43406F583C083C0829006C4B9
:10610A00E0D082D08375F00912477C7401F022A492
:10611A0024CDF582E43406F583C083C0829006C498
:0E612A00E0D082D08375F00912477CE4F022A9
:104B6600126AA09005A574FFF0A37434F0A374C074
:104B7600F09007AFE075F01DA424CAF582E4340670
:104B8600F583C083C0829006C4E0D082D08375F0DE
:104B96000912477CE07BFF60067A3479D780047A75
:104BA6003479D99005A8EBF0A3EAF0A3E9F09007D1
:104BB600AFE0FF75F01DA424C6F582E43406F58344
:104BC600C083C0829006C4E0FED082D08375F0090F
:104BD60012477CE0FD9005ABE4F0A3EDF0EF75F035
:104BE6001DA424CBF582E43406F58375F009EE1294
:104BF600477CE07BFF60067A3479DB80047A34797F
:104C0600DD9005ADEBF0A3EAF0A3E9F09007AFE085
:104C1600FF75F01DA424C7F582E43406F583C0832E
:104C2600C0829006C4E0FED082D08375F009124798
:104C36007CE0FD9005B0E4F0A3EDF0EF75F01DA467
:104C460024CCF582E43406F58375F009EE12477C30
:104C5600E07BFF60067A3479DF80047A3479E1906C
:104C660005B2EBF0A3EAF0A3E9F09007AFE075F028
:104C76001DA424C5F582E43406F583C083C0829062
:104C860006C4E0D082D08375F00912477CE075F047
:104C960003A4240FF582E5F03436F583E493F97422
:104CA6000193FA7402939005B5C9F0A3EAF0A3E95B
:104CB600F07B017A0879641248669007ADE07003CC
:104CC600024D589005A574FFF0A37434F0A374E365
:104CD600F09007AFE0FF75F01DA424CDF582E43413
:104CE60006F583C083C0829006C4E0FED082D083DE
:104CF60075F00912477CE07BFF60067A3479F7800D
:104D0600047A3479F99005A8EBF0A3EAF0A3E9F068
:104D1600EF75F01DA424C8F582E43406F58375F01A
:104D260009EE12477CE0FF9005ABE4F0A3EFF07BC1
:104D3600017A0879751248667E377F2F7D05125CE9
:104D46002C90083F7401F0A37408F0A37462F0027B
:104D56004E499005A574FFF0A37434F0A374FBF0DC
:104D66009007AFE0FF75F01DA424CDF582E434066C
:104D7600F583C083C0829006C4E0FED082D08375DE
:104D8600F00912477CE07BFF60067A3479F78004ED
:104D96007A3479F99005A8EBF0A3EAF0A3E9F0EFED
:104DA60075F01DA424C8F582E43406F58375F00970
:104DB600EE12477CE0FD9005ABE4F0A3EDF0EF7555
:104DC600F01DA424E1F582E43406F583E075F003D2
:104DD600A424FDF582E43435F583E493F974019354
:104DE600FA7402939005ADC9F0A3EAF0A3E9F09036
:104DF60007AFE075F01DA424E0F582E43406F583E0
:104E0600E075F003A4247FF582E43435F583E4935A
:104E1600F9740193FA7402939005B0C9F0A3EAF00D
:104E2600A3E9F07B017A0879751248667E377F110F
:104E36007D06125C2C90083F7401F0A37408F0A361
:104E46007461F09005A57401F0A37408F0A374755D
:0D4E5600F07B017A08796412642A025D4441
:105DC000126AA09005A574FFF0A37435F0A3740DBA
:105DD000F09007B3E0FF9005A8E4F0A3EFF07B019B
:105DE0007A0879641248669005A574FFF0A37435AB
:105DF000F0A37420F07B017A0879751248667E372B
:105E00007F487D01125C2C90083F7401F0A3740858
:105E1000F0A37463F09005A57401F0A37408F0A3D7
:0F5E20007475F07B017A08796412642A025D447C
:0D6A7C009007B6E06003025DC0124B662279
:106138000001020408100000030418000000000019
:106148001F000000000018040300000000100804ED
:1061580002010000040A0A11110000010102021CD8
:1061680000001C02020101000010100808070000CE
:0E6178000708081010000020406080A0C0FF43
:106A10007F381268B47F061268B47D0EE4FF021955
:016A2000F77E
:0568B4009005A8EFF0C3
:1068B900A2AF9202C2AF126832EF20E7F99005A8A1
:0968C900E0FF1263B3A20292AFDA
:0168D20022A3
:10683200A2AF9203C2AF75A0FFC2B6D2B5D2B77FE4
:1068420014DFFEAEA0C2B77F14DFFEA20392AFAF89
:01685200063F
:016853002222
:056ABE007F010268B435
:1063B300A2AF9203C2AF8FA07F147E00EF1F7001C4
:1063C3001EEF4E70F7C2B6C2B5D2B77E007F14EF90
:1063D3001F70011EEF4E70F7C2B77E007F14EF1FD0
:0B63E30070011EEF4E70F7A20392AF96
:0163EE00228C
:10666E00A2AF9202C2AF8FA0C2B5D2B7D2B67F147C
:10667E007E00EF1F70011EEF4E70F7C2B77E007FD7
:0E668E0014EF1F70011EEF4E70F7A20292AFC4
:01669C0022DB
:0C19F700900908E05FF04DFFF00268B4BA
:02697800AD0769
:10697A00A2AF9201C2AF126832EF20E7F9AF051257
:06698A00666EA20192AF4F
:0169900022E4
:0863EF00E0FBA3E0FAA3E0F9D2
:1063F7009005A8EBF0A3EAF0A3E9F09005A8E0FB6D
:10640700A3E0FAA3E0F912453B60179005A8A3E4BF
:1064170075F0011245EFA9F0FA12453BFF126978B2
:0364270080D922F7
:0B642A009005A2EBF0A3EAF0A3E9F05C
:10643500A2AF9200C2AF126ABEE4FDFF1269AA9034
:1064450005A21263EFE4FD7F011269AA9005A5126A
:0D64550063EF7D117F011269AAA20092AFD2
:016462002217
:1069AA00A2AF9201C2AFEF75F040A42D2480FF126E
:0669BA0068B4A20192AFD7
:0169C00022B4
:106A2100AE84E4F584EF90617E93F5D3AF068F8455
:016A31002242
:10406100000000010003000500070008000A000C21
:10407100000E000F00110013001500160018001AA1
:10408100001C001D001F0021002300240026002821
:10409100002A002B002D002F0031003200340036A1
:1040A10000380039003B003D003F00400042004421
:1040B100004600470049004B004D004E00500052A1
:1040C1000054005500570059005B005C005E006021
:1040D10000620063006500670069006A006C006EA1
:1040E100007000710073007500770078007A007C21
:1040F100007E007F00810083008500860088008AA1
:10410100008C008D008F0091009300940096009820
:10411100009A009B009D009F00A100A200A400A6A0
:1041210000A800A900AB00AD00AF00B000B200B420
:1041310000B600B700B900BB00BD00BE00C000C2A0
:1041410000C400C500C700C900CB00CC00CE00D020
:1041510000D200D300D500D700D900DA00DC00DEA0
:1041610000E000E100E300E500E700E800EA00EC20
:1041710000EE00EF00F100F300F500F600F800FAA0
:1041810000FC00FD00FF0000000A0014001F0029D0
:104191000033003E00480052005D00670071007C62
:1041A10000860090009A00A500AF00BA00C400CEBE
:1041B10000D900E300ED00F80102010C0116012114
:1041C100012B01350140014A0155015F016901746B
:1041D100017E01880193019D01A701B201BC01C6C5
:1041E10001D101DB01E501F001FA0204020E02191D
:1041F1000223022D02380242024C02570261026B75
:1042010002760280028A0295029F02AA02B402BECD
:1042110002C902D302DD02E802F202FC0307031124
:10422100031B03260330033A0345034F0359036479
:10423100036E03780383038D039703A203AC03B6D4
:1042410003C103CB03D503E003EA03F403FF00003A
:10425100009A00F401340165018E01B001CE01E83C
:1042610001FF02150228023A024A025A0268027547
:104271000282028E029902A402AF02B902C202CBEB
:1042810002D402DC02E402EC02F402FB03020309A1
:10429100030F0316031C03220328032E03340339DF
:1042A100033E03440349034E03530357035C036175
:1042B1000365036A036E03720376037A037E038246
:1042C1000386038A038E039103950399039C03A03C
:1042D10003A303A603AA03AD03B003B303B603B953
:1042E10003BC03BF03C203C503C803CB03CE03D082
:1042F10003D303D603D903DB03DE03E003E303E5C2
:1043010003E803EA03ED03EF03F203F403F603F911
:1043110003FB03FD03FF5051525456585B5F636822
:104321006E757D8793A2B3C8E1FF505255595E6601
:10433100707E91ABCEFF505154575B60666F7A89A6
:104341009CB5D5FF40002000155510000CCC0AAAE1
:1043510009240800071C0666055504920400038E13
:104361000333028F022201D40199016C014701112B
:1043710000EA00CC00B600A3008800750066005B6F
:10438100005100410036002E002800240020001BAF
:1043910000170014001200100000000C0018002487
:1043A1000030003C004800540060006C007800843C
:1043B1000090009C00A800B400C000CC00D800E42C
:1043C10000F000FC010801140120012C0138014416
:1043D1000150015D016901750181018D019901A5FD
:1043E10001B101BD01C901D501E101ED01F90205EB
:1043F1000211021D022902350241024D02590265D4
:104401000271027D0289029502A102AE02BA02C6C0
:1044110002D202DE02EA02F60302030E031A0326A7
:104421000332033E034A03560362036E037A038693
:104431000392039E03AA03B603C203CE03DA03E683
:0444410003F203FF80
:10646300E4FFEF75F008A42430F582E43404F583E7
:10647300E4F0A3F0FEEF75F008A42432F582E434CF
:1064830004F58375F002EE12477CE4F0A3F00EEE00
:08649300B403E20FEFB410CADC
:01649B0022DE
:066AA600123BF2024E63F8
:103BF2009004307420F09004387410F090044074F3
:103C020080F09004487470F09004507440F0900476
:103C1200587430F09004607460F09004687450F04E
:103C22009007AFE075F01DA424C7F582E43406F5D1
:103C320083C083C0829006C4E0D082D08375F0092D
:103C420012477CE0FFC394144005EF9428400BEF29
:103C5200C3943C407AEF945050759007AFE075F0F2
:103C62001DA424C7F582E43406F583C083C0829084
:103C720006C4E0D082D083126A42C374139FFFE469
:103C82009400FE74172FF58274433EF583E4937516
:103C9200F010A4FF900430E045F0F0A3E04FF09064
:103CA20007AFE075F01DA424C7F582E43406F5835E
:103CB200C083C0829006C4E0D082D083126A42EFF1
:103CC2009043179375F010A4FF900438023D43907F
:103CD20007AFE075F01DA424C7F582E43406F5832E
:103CE200C083C0829006C4E0D082D083126A42C3ED
:103CF20074139FFFE49400FE74172FF58274433E01
:103D0200F583E49375F010A4FF900438E045F0F0D9
:103D1200A3E04FF09007AFE075F01DA424C7F58231
:103D2200E43406F583C083C0829006C4E0D082D01A
:103D320083126A42EF9043179375F010A4FF900428
:103D420030E045F0F0A3E04FF09007AFE075F01DD2
:103D5200A424C6F582E43406F583C083C0829006AB
:103D6200C4E0D082D08375F00912477CE0FFC3948F
:103D7200144005EF9428400BEFC3943C4042EF946B
:103D820050503DEF75F01484ADF0EDFFC374139FF6
:103D9200FFE49400FE74172FF58274433EF583E42A
:103DA2009375F010A4FF900440E045F0F0A3E04FBB
:103DB200F0ED9043179375F010A4FF900448805ED5
:103DC2009007AFE075F01DA424C6F582E43406F531
:103DD20083C083C0829006C4E0D082D08375F0098C
:103DE20012477CE075F01484ADF0EDFFC374139FAD
:103DF200FFE49400FE74172FF58274433EF583E4CA
:103E02009375F010A4FF900448E045F0F0A3E04F52
:103E1200F0ED9043179375F010A4FF900440E04535
:103E2200F0F0A3E04FF09007AFE075F01DA424C8B6
:103E3200F582E43406F583C083C0829006C4E0D0E4
:103E420082D08375F00912477CE0FFC394144005C9
:103E5200EF9428400BEFC3943C4042EF9450503D06
:103E6200EF75F01484ADF0EDFFC374139FFFE4947B
:103E720000FE74172FF58274433EF583E49375F0C8
:103E820010A4FF900450E045F0F0A3E04FF0ED9055
:103E920043179375F010A4FF900458805E9007AF0B
:103EA200E075F01DA424C8F582E43406F583C083CE
:103EB200C0829006C4E0D082D08375F00912477C9C
:103EC200E075F01484ADF0EDFFC374139FFFE4942A
:103ED20000FE74172FF58274433EF583E49375F068
:103EE20010A4FF900458E045F0F0A3E04FF0ED90ED
:103EF20043179375F010A4FF900450E045F0F0A32F
:103F0200E04FF09007AFE075F01DA424C5F582E400
:103F12003406F583C083C0829006C4E0D082D08389
:103F220075F00912477CE0FFC3940C4005EF94182A
:103F32004016EFC394244005EF9430400BEFC39436
:103F42003C4043EF9448503EEF75F00C84ADF0EDE9
:103F5200FFC3740B9FFFE49400FE742B2FF5827451
:103F6200433EF583E49375F010A4FF900460E045AE
:103F7200F0F0A3E04FF0ED90432B9375F010A4FF07
:103F82009004680240589007AFE075F01DA424C564
:103F9200F582E43406F583C083C0829006C4E0FF54
:103FA200D082D08375F00912477CE0C39448900711
:103FB200AFE075F01D4048A424C5F582E43406F54F
:103FC2008375F009EF12477CE0FD9042EF9375F0A4
:103FD20010A4FF900460E045F0F0A3E04FF0EDFF85
:103FE200C374559FFFE49400FE74372FF582744327
:103FF2003EF583E49375F010A4FF9004688057A403
:1040020024C5F582E43406F583C083C0829006C4D9
:10401200E0D082D08375F00912477CE075F00C8401
:10402200ADF0EDFFC3740B9FFFE49400FE742B2FE1
:10403200F58274433EF583E49375F010A4FF900477
:1040420068E045F0F0A3E04FF0ED90432B9375F05C
:0F40520010A4FF900460E045F0F0A3E04FF022CF
:045A2000E4FFC2FAE3
:105A24009006B2E4F0A3740AF09006B274FFF5F0A5
:0E5A34001245EFFCD3E5F09400EC940050EB2B
:105A4200E59A20E7FBEF75F008A42430F582E434F0
:105A520004F583E0F59B30FFFDC2FFE59A20E7FBEA
:105A6200EF75F008A42431F582E43404F583E0F5FF
:105A72009B30FFFDC2FFE4FEE59A20E7FBEF75F0E5
:105A820008A42432F582E43404F58375F002EE12A0
:105A9200477CE0F59B30FFFDC2FFE59A20E7FBEF74
:105AA20075F008A42433F582E43404F58375F0021A
:105AB200EE12477CE0F59B30FFFDC2FF0EEEB40311
:035AC200B7D2FA5E
:105AC5009006B2E4F0A3740AF09006B274FFF5F004
:0E5AD5001245EFFCD3E5F09400EC940050EB8A
:095AE3000FEF64106003025A2267
:015AEC002297
:104E6300E49006B2F09006B2E0FFC394034003025D
:104E730050B99007B4E0600F9006C4E0FEC374021B
:104E83009E6F600302504B9006B2E0FF25E0243290
:104E9300F582E43404F5837410F0EF25E02432F551
:104EA30082E43404F583C083C082E0FCA3E0FDC345
:104EB30074029F75F008A42418F582E43404F58382
:104EC300E0FEA3E0FFD394FFEE9403400A7A0F7B46
:104ED300FC7E0F7FFC800BEF7802C333CE33CED83A
:104EE300F9FFEC4EFEED4FFFD082D083EEF0A3EF3F
:104EF300F09006B2E0FF25E0243AF582E43404F5AD
:104F0300837420F0EF25E0243AF582E43404F5833A
:104F1300C083C082E0FCA3E0FDC374029F75F00868
:104F2300A4241AF582E43404F583E0FEA3E0FFD35E
:104F330094FFEE9403400A7A007B007E007F00809A
:104F430014C374FF9FFF74039EFEEF7802C333CE36
:104F530033CED8F9FFEC4EFEED4FFFD082D083EE77
:104F6300F0A3EFF09006B2E0FF25E02442F582E4DF
:104F73003404F5837430F0EF25E02442F582E43401
:104F830004F583C083C082E0FCA3E0FDC374029FE9
:104F930075F008A4241CF582E43404F583E0FEA331
:104FA300E0FFD394FFEE9403400A7A007B007E0077
:104FB3007F008014C374FF9FFF74039EFEEF78028B
:104FC300C333CE33CED8F9FFEC4EFEED4FFFD08284
:104FD300D083EEF0A3EFF09006B2E0FF25E0244A81
:104FE300F582E43404F5837440F0EF25E0244AF5B8
:104FF30082E43404F583C083C082E0FCA3E0FDC3F4
:1050030074029F75F008A4241EF582E43404F5832A
:10501300E0FEA3E0FFD394FFEE940340067E007FFF
:10502300008014C374FF9FFF74039EFEEF7802C3D6
:1050330033CE33CED8F9FFEC4EFEED4FFFD082D006
:1050430083EEF0A3EFF080659006B2E0FF25E02445
:1050530032F582E43404F5837410F0EF25E0243A4A
:10506300F582E43404F5837420F0EF25E0243AF567
:1050730082E43404F583C083C082E0440FFFA3E0DD
:1050830044FCD082D083CFF0A3EFF09006B2E0FFD0
:1050930025E02442F582E43404F5837430F0EF25EF
:1050A300E0244AF582E43404F5837440F09006B2B8
:0650B300E004F0024E686B
:0150B90022D4
:086A420075F00912477CE0FF2A
:076A4A00EF75F01484AFF0BA
:016A51002222
:10561E00F58375F009ED12477CE025E02487F582CD
:10562E00E43441F583E493FC740193FD9004B2E0FD
:10563E00FAA3E0FB9006B87403F0A374FFF0A3E4A2
:03564E00F0A3F0D6
:085651009006B2EEF0A3EFF0A9
:10565900A9849006B2E0FEA3E0FFC3ED9FFFEC9E94
:10566900900402F0A3EFF075840375C3019004025E
:10567900E0FF3395E08FC2A3E0F5C1EAFF3395E07F
:105689008F92EBF59190040AE004F0E004F09004A5
:105699000412474B00000000900404E596F0A3E5CE
:1056A90095F0A3E594F0A3E593F0900404E0FCA33E
:1056B900E0FDA3E0FEA3E0FF780F1246E4900404A6
:1056C90012473F900406E0FFA3E0900408CFF0A33F
:1056D900EFF0AF018F849006B2E0FEA3E0FF9004E3
:1056E90009E02FF0900408E03EF09006BAE0FEA32E
:1056F900E0FF900409E02FF0900408E03EF09006E6
:10570900B8E0FEA3E0FF900408E0FCA3E0D39FEE1D
:105719006480F8EC648098400122C3EC6480948032
:0E5729005004E4FEFF22900408E0FEA3E0FF1F
:01573700224F
:0468D3007DFF7C03C6
:0E68D7009006B2EEF0A3EFF0A3ECF0A3EDF00C
:0C68E5009006B3E02BFF9006B2E03AFEF4
:0168F1002284
:031A2D00021A3961
:101A3900C0E0C0F0C083C082C0D075D000C000C073
:0D1A490001C002C003C004C005C006C007F4
:101A56009006ADE584F0758402E5E854019008F738
:101A6600F053E8FE43E70475BB03C2EDD2EC30ED5C
:101A7600FD9006AFE5BEF09008F7E060109006AF67
:101A8600E0C394EF50079004B6E4F080059008F7A1
:101A9600E4F09006AFE0C3941F5002E4F0758400B2
:101AA6009007AEE070030228E09007ADE0700302F5
:021AB6001BD83B
:101AB8007F071267C69004B4EEF0A3EFF090040E0F
:101AC800E0FF9007B0E06F6019E0FBFD7C007E0F3F
:101AD8007FFF12459A90040BEEF0A3EFF090040EEE
:101AE800EBF090040BE0FCA3E0FD9004B4E0FAA353
:101AF800E0FBFFAE0212459AEF049007B1F0D394D1
:101B08000740037407F09007B1E0FF14900415F044
:101B180090040DE0FEEF6E600A9007B1E090040DAE
:101B2800F08026C3EA9401500B90040FE0FEC3EE48
:101B3800940150159004B4E0FEC3EE940140109057
:101B4800040FE0FEEE940150069007B97401F0907E
:101B5800040BE0FCA3E0FD9004B4E0FEA3E0FF1258
:101B6800459AAE04AF05E4FCFD9006BF12473F90CE
:101B780006BFE0FCA3E0FDA3E0FEA3E0FF780F12A0
:101B880046F79006BF12473F9006BFE0FCA3E0FD72
:101B9800A3E0FEA3E0FFC004C005C006C007900490
:101BA8000BE0FEA3E0FFE4F8F9AA06AB07D007D0E4
:101BB80006D005D0041246419006BF12473F900454
:0D1BC800B4E0FFA3E090040FCFF0A3EFF016
:101BD500021E3C9008F7E060449007B1E075F01DE7
:101BE500A424E1F582E43406F583E0FF6403602D67
:101BF500EF640460289006BFE0FCA3E0FDA3E0FECF
:101C0500A3E0FF9004B012473F9006BF12474B0078
:101C15000000009007B97401F0900416F09007B128
:101C2500E075F01DA424E1F582E43406F583E0FFB8
:101C3500B401069006AFE0702BEFB402069006AF34
:101C4500E060219007B1E075F01DA424E1F582E480
:101C55003406F583E0FF64036004EFB4040F9004D9
:0D1C6500B6E06009900416E07003021E371F
:101C72007F071267C69006B0EEF0A3EFF09004164D
:101C8200E060059006E080119007B1E075F01DA4B8
:101C920024E0F582E43406F583E025E02445F5826C
:101CA200E43443F583E493FE740193FFE4FCFD9076
:101CB200041112473F900411E0FCA3E0FDA3E0FEF3
:101CC200A3E0FFC004C005C006C0079006B0E0FE56
:101CD200A3E0FF7C007D09124588EEC4540F240165
:101CE200FFE433FEE4F8F9AA06AB07D007D006D02A
:101CF20005D00412464190041112473FE4FFFEFD55
:101D0200FC900411E0F8A3E0F9A3E0FAA3E0FBC31E
:101D12001246D3700A90041112474B000000019042
:101D220006BFE0FCA3E0FDA3E0FEA3E0FF900411E8
:101D3200E0F8A3E0F9A3E0FAA3E0FBEF2BFFEE3A11
:101D4200FEED39FDEC38FC9006BF12473FE47FFF01
:101D52007E7FFDFC9006BFE0F8A3E0F9A3E0FAA3C2
:101D6200E0FBD31246D35003021E1E900416E0601D
:101D7200059007B1E4F09007B1E075F01DA424E1ED
:101D8200F582E43406F583E0FF64036004EFB404F3
:101D9200179008F7E070119004B604F09006BF1295
:101DA200474B00007FFF80749007B1E004F090077A
:101DB200B0E0FF9007B1E0D39F4002E4F09007B19A
:101DC200E075F01DA424E1F582E43406F583E0FF1A
:101DD200B401069006AFE0700AEFB402129006AFAB
:101DE200E0700C9006BF12474B0000000080239069
:101DF20006BFE0FCA3E0FDA3E0FEA3E0C39400FF66
:101E0200EE9480FEED9400FDEC9400FC9006BF126F
:101E1200473F900416E4F09007B904F09007B1E050
:101E220014FF9007B0E0FEEFD39E4004AF0680009F
:051E3200900415EFF023
:101E37009008F7E4F0900416E0700302230B900675
:101E4700AEE4F09006AEE0FFC394034003022A829B
:101E5700EF75F009A424CCF582E43406F583E0603D
:101E67005A9006AEE075F009A424C5F582E434065D
:101E7700F583E025E02499F582E43443F583E49380
:101E8700FC740193FDC004C005EF75F003A424F8AA
:101E9700F582E43408F583E0FF12650E9006BAEE8A
:101EA700F0A3EFF09006B87403F0A374FFF0D00529
:101EB700D004FB7A7FE4FFFE021F80900415E075D3
:101EC700F01DA424C5F582E43406F583C083C082DF
:101ED7009006AEE0FDD082D08375F00912477CE012
:101EE70025E02499F582E43443F583E493FE7401F5
:101EF70093FF9007B1E075F01DA424C5F582E43483
:101F070006F58375F009ED12477CE025E02499F585
:101F170082E43443125631C006C0079006AEE0FF94
:101F270075F009A424C5F582E43406F583E025E0BD
:101F37002499F582E43443F583E493FC740193FD1B
:101F4700C004C005EF75F003A424F8F582E4340853
:101F5700F583E0FF12650E9006BAEEF0A3EFF0905E
:101F670006C1E0FAA3E0FB9006B87403F0A374FF80
:101F7700F0D005D004D007D0061256519006AEE037
:101F870075F008A42418F582E43404F583EEF0A371
:101F9700EFF09006AEE0FF75F009A424CDF582E4DA
:101FA7003406F583E06039EF75F009A424C8F5829B
:101FB700E43406F583E025E02487F582E43441F52F
:101FC70083E493FC740193FD9006B87403F0A37443
:101FD700FFF0A3E4F0A3F07BFF7A7FFFFE02206B04
:101FE700900415E075F01DA424C8F582E43406F5C5
:101FF70083C083C0829006AEE0FDD082D08375F0A7
:102007000912477CE025E02487F582E43441F58313
:10201700E493FE740193FF9007B1E075F01DA424CB
:10202700C8F582E4340612561E9006AEE075F00934
:10203700A424C8F582E43406F583E025E02487F577
:1020470082E43441F583E493FC740193FD9006C167
:10205700E0FAA3E0FB9006B87403F0A374FFF0A3C3
:10206700E4F0A3F01256519006AEE075F008A424F0
:102077001EF582E43404F583EEF0A3EFF09006AE8C
:10208700E0FF75F009A424CAF582E43406F583E07D
:102097006057EF75F009A424C6F582E43406F5838A
:1020A700E025E02487F582E43441F583E493FC746A
:1020B7000193FDC004C005EF75F003A424FAF5826F
:1020C700E43408F583E0FF1261869006BAEEF0A3C8
:1020D700EFF09006B87403F0A374FFF0D005D004B6
:1020E700FB7A7FE4FFFE02219B900415E075F01D4B
:1020F700A424C6F582E43406F583C083C082900623
:10210700AEE0FDD082D08375F00912477CE025E070
:102117002487F582E43441F583E493FE740193FF49
:102127009007B1E075F01DA424C6F582E4340612C9
:10213700561EC006C0079006AEE0FF75F009A4243E
:10214700C6F582E43406F583E025E02487F582E4CA
:102157003441F583E493FC740193FDC004C005EF9B
:1021670075F003A424FAF582E43408F583E0FF123E
:1021770061869006BAEEF0A3EFF09006C1E0FAA3ED
:10218700E0FB9006B87403F0A374FFF0D005D00409
:10219700D007D0061256519006AEE075F008A42479
:1021A7001AF582E43404F583EEF0A3EFF09006AE5F
:1021B700E0FF75F009A424CBF582E43406F583E04B
:1021C7006066EF75F009A424C7F582E43406F58349
:1021D700E025E02487F582E43441F583E493FC7439
:1021E7000193FDC004C005EF75F003A424F9F5823F
:1021F700E43408F583E0FF12650EC006C0077F03CD
:1022070012650ED0E02FFFD0E03E9006BAF0A3EFA4
:10221700F09006B87403F0A374FFF0D005D004FB68
:102227007A7FE4FFFE0222E9900415E075F01DA411
:1022370024C7F582E43406F583C083C0829006AED6
:10224700E0FDD082D08375F00912477CE025E024B9
:1022570087F582E43441F583E493FE740193FF909C
:1022670007B1E075F01DA424C7F582E434061256C1
:102277001EC006C0079006AEE0FF75F009A424C78C
:10228700F582E43406F583E025E02487F582E4341B
:1022970041F583E493FC740193FDC004C005EF7519
:1022A700F003A424F9F582E43408F583E0FF12650E
:1022B7000EC006C0077F0312650ED0E02FFFD0E0E7
:1022C7003E9006BAF0A3EFF09006C1E0FAA3E0FB58
:1022D7009006B87403F0A374FFF0D005D004D007BC
:1022E700D0061256519006AEE075F008A4241CF5EE
:1022F70082E43404F583EEF0A3EFF09006AEE00439
:10230700F0021E4A9006AEE4F09006AEE0FFC394DA
:10231700034003022A829007B1E0FD75F01DA42453
:10232700CCF582E43406F58375F009EF12477CE0BB
:1023370090041570030223D9E075F01DA424C5F598
:1023470082E43406F583C083C0829006AEE0FCD0F9
:1023570082D08375F00912477CE025E02499F58245
:10236700E43443F583E493FE740193FFC006C0078A
:10237700ED75F01DA424C5F582E43406F58375F0E8
:1023870009EC12477CE025E02499F582E43443F513
:1023970083E493FC740193FDC004C0059006AEE08E
:1023A70075F003A424F8F582E43408F583E0FF12FE
:1023B700650E9006BAEEF0A3EFF09006B87403F03E
:1023C700A374FFF0D005D004D007D006FB7A7F02B4
:1023D7002478E075F01DA424C5F582E43406F5835E
:1023E700C083C0829006AEE0FDD082D08375F0092D
:1023F70012477CE025E02499F582E43443F583E431
:1024070093FE740193FFC006C0079007B1E075F013
:102417001DA424C5F582E43406F58375F009ED1291
:10242700477CE025E02499F582E43443F583E4937F
:10243700FC740193FDC004C0059006AEE075F0037F
:10244700A424F8F582E43408F583E0FF12650E90C2
:1024570006BAEEF0A3EFF09006C1E0FAA3E0FB9016
:1024670006B87403F0A374FFF0D005D004D007D0EA
:10247700061256519006AEE075F008A42418F582AE
:10248700E43404F583EEF0A3EFF09007B1E0FD75B7
:10249700F01DA424CDF582E43406F583C083C08201
:1024A7009006AEE0D082D08375F00912477CE090A9
:1024B70004156071E075F01DA424C8F582E43406A4
:1024C700F583C083C0829006AEE0FCD082D08375CE
:1024D700F00912477CE025E02487F582E43441F5D2
:1024E70083E493FE740193FFED75F01DA424C8F5F2
:1024F70082E43406F58375F009EC12477CE025E0A9
:102507002487F582E43441F583E493FC740193FD59
:102517009006B87403F0A374FFF0A3E4F0A3F07B74
:10252700FF7A7F8076E075F01DA424C8F582E43435
:1025370006F583C083C0829006AEE0FDD082D083CB
:1025470075F00912477CE025E02487F582E43441E1
:10255700F583E493FE740193FF9007B1E075F01DD6
:10256700A424C8F582E43406F58375F009ED124713
:102577007CE025E02487F582E43441F583E493FC8D
:10258700740193FD9006C1E0FAA3E0FB9006B874CE
:1025970003F0A374FFF0A3E4F0A3F01256519006E2
:1025A700AEE075F008A4241EF582E43404F583EE4A
:1025B700F0A3EFF09007B1E0FD75F01DA424CAF574
:1025C70082E43406F583C083C0829006AEE0D082F1
:1025D700D08375F00912477CE0900415700302263A
:1025E70082E075F01DA424C6F582E43406F583C0A5
:1025F70083C0829006AEE0FCD082D08375F00912CA
:10260700477CE025E02487F582E43441F583E493B1
:10261700FE740193FFC006C007ED75F01DA424C624
:10262700F582E43406F58375F009EC12477CE02562
:10263700E02487F582E43441F583E493FC74019345
:10264700FDC004C0059006AEE075F003A424FAF5BA
:1026570082E43408F583E0FF1261869006BAEEF053
:10266700A3EFF09006B87403F0A374FFF0D005D081
:1026770004D007D006FB7A7F022721E075F01DA45E
:1026870024C6F582E43406F583C083C0829006AE83
:10269700E0FDD082D08375F00912477CE025E02465
:1026A70087F582E43441F583E493FE740193FFC018
:1026B70006C0079007B1E075F01DA424C6F582E4B3
:1026C7003406F58375F009ED12477CE025E0248791
:1026D700F582E43441F583E493FC740193FDC0046F
:1026E700C0059006AEE075F003A424FAF582E43441
:1026F70008F583E0FF1261869006BAEEF0A3EFF0CB
:102707009006C1E0FAA3E0FB9006B87403F0A37447
:10271700FFF0D005D004D007D0061256519006AE70
:10272700E075F008A4241AF582E43404F583EEF08A
:10273700A3EFF09007B1E0FD75F01DA424CBF5825F
:10274700E43406F583C083C0829006AEE0D082D021
:102757008375F00912477CE0900415700302281076
:10276700E075F01DA424C7F582E43406F583C08321
:10277700C0829006AEE0FCD082D08375F009124784
:102787007CE025E02487F582E43441F583E493FE79
:10279700740193FFC006C007ED75F01DA424C7F5AB
:1027A70082E43406F58375F009EC12477CE025E0F6
:1027B7002487F582E43441F583E493FC740193FDA7
:1027C700C004C0059006AEE075F003A424F9F582B5
:1027D700E43408F583E0FF12650EC006C0077F03E7
:1027E70012650ED0E02FFFD0E03E9006BAF0A3EFBF
:1027F700F09006B87403F0A374FFF0D005D004D0AE
:1028070007D006FB7A7F0228BEE075F01DA424C717
:10281700F582E43406F583C083C0829006AEE0FDFE
:10282700D082D08375F00912477CE025E02487F534
:1028370082E43441F583E493FE740193FFC006C03C
:10284700079007B1E075F01DA424C7F582E43406AC
:10285700F58375F009ED12477CE025E02487F582C2
:10286700E43441F583E493FC740193FDC004C0058F
:102877009006AEE075F003A424F9F582E43408F578
:1028870083E0FF12650EC006C0077F0312650ED0F6
:10289700E02FFFD0E03E9006BAF0A3EFF09006C11C
:1028A700E0FAA3E0FB9006B87403F0A374FFF0D03E
:1028B70005D004D007D0061256519006AEE075F049
:1028C70008A4241CF582E43404F583EEF0A3EFF0AA
:1028D7009006AEE004F00223109006AEE4F09007F5
:1028E700AFE075F01DA424C5F582E43406F583C076
:1028F70083C0829006AEE0FDD082D08375F00912C6
:10290700477CE025E02499F582E43443F583E4939A
:10291700FE740193FFC006C007ED75F003A424F809
:10292700F582E43408F583E0FF12650EAA06AB07CB
:10293700D007D0061268D39006AEE0FD75F008A464
:102947002418F582E43404F583EEF0A3EFF0900742
:10295700AFE075F01DA424C8F582E43406F583754D
:10296700F009ED12477CE025E02487F582E4344145
:10297700F583E493FE740193FFE4FBFA7DFF12688D
:10298700D79006AEE0FD75F008A4241EF582E43466
:1029970004F583EEF0A3EFF09007AFE075F01DA408
:1029A70024C6F582E43406F58375F009ED12477CF9
:1029B700E025E02487F582E43441F583E493FE744F
:1029C7000193FFC006C007ED75F003A424FAF58252
:1029D700E43408F583E0FF126186AA06AB07D00747
:1029E700D0061268D39006AEE0FD75F008A4241A4D
:1029F700F582E43404F583EEF0A3EFF09007AFE03F
:102A070075F01DA424C7F582E43406F58375F00933
:102A1700ED12477CE025E02487F582E43441F58315
:102A2700E493FE740193FFC006C007ED75F003A49D
:102A370024F9F582E43408F583E0FF12650EC00639
:102A4700C0077F0312650ED0E02FFBD0E03EFAD01F
:102A570007D0061268D39006AEE075F008A4241CD0
:102A6700F582E43404F583EEF0A3EFF09006AEE0D0
:102A770004F0E0C3940350030228E5126463126A6A
:0F2A8700A6125A20758401C2CF9006ADE0F584E7
:102A9600D007D006D005D004D003D002D001D00094
:0B2AA600D0D0D082D083D0F0D0E0323E
:1065B0009008F87404F09008FB04F09008FE04F0D2
:1065C000E49008F9F09008FC04F09008FF04F090C3
:1065D00008FA7405F09008FD04F090090004F02218
:10650E00AD84E4F5848FBBC2EDD2EC30EDFD900688
:10651E00B2E5BFF0A3E5BEF09006B2E0FEA3E078D0
:10652E0002CEC313CE13D8F9F0EE9006B2F0AF053B
:07653E008F84E0FEA3E0FFE3
:016545002233
:1067C600AE84E4F5848FBBC2EDD2EC30EDFD9006CD
:1067D600B2E5BFF0A3E5BEF0AF068F849006B2E047
:0467E600FEA3E0FF2F
:0167EA00228C
:10618600AD84ACE775840253E7FBE5E85401FB8F69
:10619600BBC2EDD2EC30EDFDE49006B2F0A3E5BE55
:1061A600F09006B2E0FEA3E07802C333CE33CED839
:1061B600F9F0EE9006B2F053E8FEAF03EB42E8AF1B
:0C61C600048FE7AF058F84E0FEA3E0FF2C
:0161D20022AA
:031A090002674F22
:10674F00C0E0C083C082C0D0900417E05407C39448
:10675F0004500A9004B6E4F09008F704F0C28BD00E
:08676F00D0D082D083D0E032CB
:031A330002649CAE
:0D649C00C0E0C083C082C0D075D000C00732
:1064A900AF8475840275BB03C2EDD2EC30EDFD906B
:1064B90006BCE5BEF0E5E830E00353E7FBC2CF8F49
:0164C900844E
:0B64CA00D007D0D0D082D083D0E032C9
:031A3600026AC37E
:046AC30053E7F33270
:1061D3009006A1E584F0A2AF9200AF01AE027C006D
:1061E300E4FDA312473F9006A4E0FEA3E07812A6C5
:1061F3000608F6E4F584C2AF43B701438F02438F29
:106203000118E6FE08E6F5828E83E4F053B7FEF547
:0B6213008FA20092AF9006A1E0F5847E
:01621E00225D
:055EF8009006A7EDF08B
:105EFD00A3E584F0A2AF9200AF01AE027C00E4FDF9
:105F0D00A312473F9006A7E0FFFD3395E0FCEDF4AB
:105F1D004C60299006ABE0FCA3E07812A60408F6CD
:105F2D00E4F584C2AF43B701758F0118E6FC08E6AE
:105F3D00F5828C83EFF053B7FEE4F58FA20092AF9C
:065F4D009006A8E0F584B7
:015F5300222B
:105E2F009006A1EEF0A3EFF0A3ECF0A3EDF0A3EA40
:105E3F00F0A3EBF09006A5E07002A3E06046900699
:105E4F00A1E0FEA3E0AA06F97B01A3E0FEA3E0F523
:105E5F00828E83E0FD125EF89006A6E024FFF0909C
:105E6F0006A5E034FFF09006A4E004F0700690065B
:105E7F00A3E004F09006A2E004F070B89006A1E051
:055E8F0004F080B022C8
:086A8900E4900000F0A3F022EC
:10672600900000E0FEA3E0AA06F97B011261D39077
:106736000000E0FEA3E0FF7C007D021B7A04125EEF
:096746002FE4900000F0A3F02202
:0D5B960090069CEDF090069AEEF0A3EFF063
:105BA300EE54FCFE900000E0FCA3E0FD7002EE6CFE
:105BB3006059ED4C600312672690069AE0FEEE549E
:105BC300FCFE7F00900000F0A3EFF090069DEEF046
:105BD300A3EFF0A37400F0A37402F07FFF7E0390A1
:105BE300069DE475F0011245EF85F082F583E49399
:105BF300FD90069FE475F0011245EF85F082F58371
:105C0300EDF0EF1F70011EEF4E70D490069CE0FF85
:105C130090069AE0FCA3E0FDEC5403FC74022DF51E
:085C23008274003CF583EFF0F0
:015C2B002256
:1062B2009005A4EEF0A3EFF0A3ECF0A3EDF0A3EAB7
:1062C200F0A3EBF09005A874FFF5F01245EF45F04E
:1062D20060239005A4E475F0011245EFAFF0FE9043
:1062E20005A6E475F0011245EF85F082F583E0FD25
:0662F200125B9680CF2232
:106874009005A2EFF0A3EDF07F0A125AED9005A265
:10688400E0FF125AED9005A3E0FF125AED026A6E82
:086A91007F02125AED026A6E49
:0665E000126AB2EF602711
:1065E6009005A27409F0A37401F01265469005A205
:1065F600E475F0011245EF85F082F583EFF0126A3B
:07660600B8EF70E67F0122EE
:03660D007F0022E9
:1069C1009005A2EFF07F2F125AED9005A2E0FF1281
:0569D1005AED026A6EA0
:1069D6009005A2EFF07F30125AED9005A2E0FF126B
:0569E6005AED026A6E8B
:011A1700FFCF
:05626A009005A2EFF019
:10626F00126A89E49005A3F09005A2E0FFA3E0FE77
:10627F00C39F502375F0EBEEA42401F582E5F034B3
:10628F0080AF82FE7C067DC57BEB7A001262B290F6
:10629F0005A3E004F080D17E807F007D01125B9624
:0362AF000267265D
:101A1B00126A897E807F009007B3E0FD125B96020D
:021A2B0067262C
:10692C007B017A0679C59005A612474B000000EB57
:0A693C00E4FD1267777F1E02626A15
:1069FE009007BBE0700374FFF0200903126A91D276
:026A0E0009225B
:031A06000269FE74
:10689400901A17E493600F12692C7E1A7F17E4FD97
:1068A400125B96126726908000E4939007B3F0225F
:10669D00A2AF9200C2AF900909E075F0EBA42401FE
:1066AD00F9748035F0FA7BFF78C57C067D017E009C
:0E66BD007FEB124515126339C209A20092AF9D
:0166CB0022AC
:1067EB00126A89900909E075F0EBA42401F582E5A2
:1067FB00F03480AF82FE7C067DC57BEB7A001262A3
:04680B00B202672648
:066AAC001267EBC2092293
:076A9900300A03126AAC226F
:10633900E49007B0F09007B0E0FFC394085021EF54
:1063490075F01DA424E1F582E43406F583E0FF64C9
:1063590004600DEF640560089007B0E004F080D593
:0D6369009007B0E0C3940840037407F022D1
:0A52F5009005A3EDF09005A2EFF084
:1052FF00D39B50030253D3E024FFFEE434FF900509
:10530F00A7F0A3CEF0EB149005A6F09005A3E02430
:10531F00FFFFE434FFFE9005A7E0FCA3E0FDD39F61
:10532F00EE6480F8EC64809840030254A4908001EE
:10533F0075F0EBED12477CEC75F0EBA42583AF8293
:10534F009005AEF0A3EFF09005A6E075F0EBA42466
:10535F0001F9748035F0FA9005AB74FFF0A3EAF011
:10536F00A3E9F0E49005A9F0A3F09005ABA3E475D1
:10537F00F0011245EFFEAFF09005AEE475F00112AB
:10538F0045EF85F082F583E493FD125B969005AAB5
:10539F00E004F070069005A9E004F0C39005AAE0C0
:1053AF0094EB9005A9E0940040C01267269005A8E1
:1053BF00E004F070069005A7E004F09005A6E00465
:1053CF00F002531A9005A3E024FFFEE434FF90058A
:1053DF00A7F0A3CEF09005A5E014A3F09005A2E0EE
:1053EF0024FFFFE434FFFE9005A7E0FCA3E0FDC31C
:1053FF009FEE6480F8EC64809850030254A4908070
:10540F000175F0EBED12477CEC75F0EBA42583AF43
:10541F00829005AEF0A3EFF09005A6E075F0EBA437
:10542F002401F9748035F0FA9005AB74FFF0A3EA0C
:10543F00F0A3E9F0E49005A9F0A3F09005ABA3E485
:10544F0075F0011245EFFEAFF09005AEE475F00177
:10545F001245EF85F082F583E493FD125B9690057C
:10546F00AAE004F070069005A9E004F0C39005AA25
:10547F00E094EB9005A9E0940040C01267269005D8
:10548F00A8E024FFF09005A7E034FFF09005A6E018
:05549F0014F00253EBC4
:0154A40022E5
:05189A009005A3EDF034
:10189F00EF14900696F0EB14A3F09005A3E014FF5D
:1018AF00900696E0D39F40030219F6A3E075F0EB84
:1018BF00A42401F582E5F03480AF82FEE49006980F
:1018CF00F0A3F00FEFAC0670010E14F5828C83E4D9
:1018DF0093FD900699E024ABF582E43405F583ED92
:1018EF00F0900699E004F07006900698E004F090EE
:1018FF000698E07004A3E064EB70C8900697E0755B
:10190F00F0EBA42401F9748035F0FA9005A674FF6A
:10191F00F0A3EAF0A3E9F0900696E075F0EBA424AB
:10192F0001F582E5F03480AF829005A9F0A3EFF0C6
:10193F00E4900698F0A3F09005A6A3E475F00112C9
:10194F0045EFFEAFF09005A9E475F0011245EF8564
:10195F00F082F583E493FD125B96900699E004F014
:10196F007006900698E004F0C3900699E094EB900F
:10197F000698E0940040C0900696E075F0EBA42422
:10198F0001F9748035F0FA9005A674FFF0A3EAF020
:10199F00A3E9F0E4900698F0A3F09005A6A3E475F0
:1019AF00F0011245EFFEAFF0900699E024ABF582FF
:1019BF00E43405F583E0FD125B96900699E004F0A0
:1019CF007006900698E004F0C3900699E094EB90AF
:1019DF000698E0940040C3126726900696E004F044
:0719EF00A3E004F00218A9B7
:0119F60022CE
:075738009005A2EBF0AC07A5
:10573F00A2AFE433A3F0AF05A3E4F0A3EFF0E07F53
:10574F0000FE9005A4F0A3EFF0AD04EDFF9005A4CB
:10575F00EEF0A3EFF0C2AF9005ACE5C0F0A3E5CF3C
:10576F00F0A3E5C3F0A3E584F0E4F58475C04075BC
:10577F00CF8F43C301900909740FF0126A89900902
:10578F0009E075F0EBA42401F9748035F0FA900567
:10579F00A874FFF0A3EAF0A3E9F0E49005A6F0A344
:1057AF00F09005A5E0FF9005A4E0FD9005A2E0FBB9
:1057BF00E49005B3F0D2001259409005ABEFF0FD25
:1057CF009005A8A3E475F0011245EFFEAFF0125B50
:1057DF00969005A5E004F070069005A4E004F09003
:1057EF0005A7E004F070069005A6E004F0C390054D
:1057FF00A7E094EB9005A6E0940040A512672690D1
:10580F000909E004F0E0C3941E500302578A900583
:10581F00AFE0F5849005ACE0F5C0A3E0F5CFA3E0D1
:10582F00F5C3C2C6126376D2C61263769005A3E0A3
:04583F0024FF92AF01
:015843002242
:075844009005A2EBF0AC0798
:10584B00A2AFE433A3F0AF059005A6E4F0A3EFF00D
:10585B00E07F00FE9005A6F0A3EFF0AD04EDFF9006
:10586B0005A6EEF0A3EFF0C2AF9005AAE5C0F0A33A
:10587B00E5CFF0A3E5C3F0A3E584F0E4F58475C0B0
:10588B004075CF8F43C301900909740FF09009093C
:10589B00E0FFC3941E507A75F0EBEFA42401F58260
:1058AB00E5F03480AF829005A8F0A3EFF0E490050B
:1058BB00A4F0A3F09005A7E0FF9005A6E0FD9005EE
:1058CB00A2E0FB9005A8E475F0011245EF85F0828C
:1058DB00F583E4939005B3F0C2001259409005A7ED
:1058EB00E004F070069005A6E004F09005A5E00436
:1058FB00F070069005A4E004F0C39005A5E094EBCE
:10590B009005A4E0940040AC900909E004F0025823
:10591B00989005ADE0F5849005AAE0F5C0A3E0F5FD
:10592B00CFA3E0F5C3C2C6126376D2C69005A3E03F
:04593B0024FF92AF04
:01593F002245
:0A5FA2004108C9004108E200C10CEB
:10699100AF84E4F58475C04475CF78C2C343E60281
:0869A10043F60275C3038F8465
:0169A90022CB
:106376007E087FCE9008C5EEF0A3EFF09008CAEE37
:10638600F0A3EFF09008C1EEF0A3EFF07E087FE3F4
:106396009008C7EEF0A3EFF09008CCEEF0A3EFF074
:0D63A6009008C3EEF0A3EFF0C20B02699166
:1064D5009008CAE475F0011245EF85F082F583EF67
:1064E500F09008CAE475F0011245EF85F082F58356
:1064F500EDF09008CAE0B4080FA3E0B4E20A9008F2
:09650500CA7408F0A374CEF02260
:0D6A6E00AF84E4F584C20BC2C4D2C58F848E
:016A7B0022F8
:105AED00200B55D20B9008CCE475F0011245EF85D3
:105AFD00F082F58374FFF07C087DF79008CCE0B55B
:105B0D00040FA3E0B5050A9008CC7408F0A374E364
:105B1D00F09008CCE475F0011245EF85F082F58325
:105B2D00E4F09008CCE0B5040FA3E0B5050A9008A9
:105B3D00CC7408F0A374E3F09008CCE475F0011276
:105B4D0045EF85F082F583E4F09008CCE0B4080FC2
:105B5D00A3E0B4F70A9008CC7408F0A374E3F090B6
:105B6D0008CCE475F0011245EF85F082F583EFF076
:105B7D009008CCE0B4080FA3E0B4F70A9008CC74F9
:095B8D0008F0A374E3F07F01228B
:1066FA009008C5E0FCA3E0FD9008C1E0B50408A33A
:10670A00E0B505037F00229008C5E0FCA3E0F5820E
:0C671A008C83E0B507037F01227F002282
:106546009008C6E004F070069008C5E004F09008D4
:10655600C5E475F0011245EF85F082F583E0FF9002
:1065660008C5E0B4080FA3E0B4E20A9008C57408B1
:05657600F0A374CEF05B
:01657B0022FD
:066AB2007FFF1266FA22CC
:066AB800E4FF1266FA2261
:031A18000250BABF
:1050BA00C0E0C0F0C083C082C0D075D000C000C0BC
:1050CA0004C005C006C007E5C154F812478852B1AA
:1050DA000051150851151051631851AF2051BC28C1
:1050EA005247305253385264505264585277605281
:1050FA006668527770526678526480528688526423
:10510A00905286985299A0000052DEC2C59008C4F7
:10511A00E004F070069008C3E004F07E087FF79080
:10512A0008C3E0B5060FA3E0B5070A9008C37408E0
:10513A00F0A374E3F09008C3E475F0011245EF851B
:10514A00F082F583E0F5C29008C3E06E7003A3E035
:10515A006F60030252DE02523A9008C4E004F07013
:10516A00069008C3E004F07E087FF79008C3E0B514
:10517A00060FA3E0B5070A9008C37408F0A374E306
:10518A00F09008C3E475F0011245EF85F082F583CB
:10519A00E0F5C29008C3E06E7003A3E06F600302FB
:1051AA0052DE02523A9008C7E0FFA3E09008C3CF4C
:1051BA00801B9008CCE0FEA3E0FF9008C3E0FCA3AC
:1051CA00E0FDB50713ECB5060F9008C7EEF0A3EFA4
:1051DA00F0C2C5D2C40252DE8D828C83E0B4FF07CE
:1051EA00C2C4D2C50252DE9008C4E004F070069030
:1051FA0008C3E004F07E087FF79008C3E0B5060F05
:10520A00A3E0B5070A9008C37408F0A374E3F0900A
:10521A0008C3E475F0011245EF85F082F583E0F5E5
:10522A00C29008C3E06E7003A3E06F60030252DE0F
:10523A009008C37408F0A374E3F00252DE9008C722
:10524A00E0FFA3E09008C3803D9008C7E0FFA3E019
:10525A009008C3CFF0A3EFF0807A80179008C7E0D8
:10526A00FFA3E09008C3CFF0A3EFF0D20CADC27F4A
:10527A00FF8004ADC2E4FF1264D580589008C1E0F3
:10528A00FFA3E09008CACFF0A3EFF0D2C480459004
:10529A0008CAE0FFA3E09008C1CFF0A3EFF0300CFA
:1052AA0033D2C5C20C802D9008C7E0FEA3E0FF9060
:1052BA0008C3EEF0A3EFF09008C1E0FDA3E0900868
:1052CA00CACDF0A3EDF0D2C4A3E06E7003A3E06FE1
:1052DA006002D2C5C2C3D007D006D005D004D00020
:0B52EA00D0D0D082D083D0F0D0E032D2
:056777009005A5EDF006
:10677C00AF01AB079005A674FF12470CEC4D4E4FC2
:10678C0060109005A5E08B828A83F00BBB00010A98
:02679C0080E299
:01679E0022D8
:03000000021800E3
:03000300021A03DB
:03000B00021A06D0
:03001300021A09C5
:03001B00021A0CBA
:03002300021A0FAF
:03002B00021A12A4
:03003300021A1599
:03003B00021A188E
:03004300021A1B83
:03004B00021A1E78
:03005300021A216D
:03005B00021A2462
:03006300021A2757
:03006B00021A2A4C
:03007300021A2D41
:03007B00021A3036
:03008300021A332B
:03008B00021A3620
:03009300021A3915
:03009B00021A3C0A
:0300A300021A3FFF
:10180000787FE4F6D8FD9000007F007E20E4F0A30E
:0A181000DFFCDEFA75812102185595
:075940009005B0EFF0A9058E
:10594700C20120C3FD20C5FAC2C4D2C5E4FFFD30A1
:10595700C3FD30C3FDE5C154F8FC64086004ECB432
:105967001013EFB40105EB44018003EB54FEF5C2BD
:105977007D01025A0EECB4180B89C27D02C2C4C263
:10598700C5025A0EECB420028045EC6428703CED49
:10599700B4020E9005B0E0F5C27D03C2C5C2C48053
:1059A70066EDB4031B300008D2C57F01C2C480571F
:1059B7009005B3E0F5C2C2C57D04E4FFC2C48047C9
:1059C700ED64047042D2C47D05803CECB4300AD249
:1059D700C4D2C57D08E4FF802EECB438028024ECE5
:1059E700B44006C2C2C2C5801EECB448028014ECA3
:1059F700B450028004ECB4580AD2C47D07AEC2C2C8
:105A0700C28004D2C4D2C5C2C3ED64076008ED6486
:085A1700056003025959AF06B6
:015A1F002264
:10181A00022AB1E493A3F8E493A34003F68001F209
:10182A0008DFF48029E493A3F85407240CC8C333CF
:10183A00C4540F4420C8834004F456800146F6DF9E
:10184A00E4800B0102040810204080905F54E47E7B
:10185A00019360BCA3FF543F30E509541FFEE49393
:10186A00A360010ECF54C025E060A840B8E493A35A
:10187A00FAE493A3F8E493A3C8C582C8CAC583CA85
:10188A00F0A3C8C582C8CAC583CADFE9DEE780BE3D
:015FAC0000F4
:10444500E709F608DFFA8046E709F208DFFA803E59
:1044550088828C83E709F0A3DFFA8032E309F60846
:10446500DFFA8078E309F208DFFA807088828C83AE
:10447500E309F0A3DFFA806489828A83E0A3F60862
:10448500DFFA805889828A83E0A3F208DFFA804C3C
:1044950080D280FA80C680D4806980F28033801013
:1044A50080A680EA809A80A880DA80E280CA80337C
:1044B50089828A83ECFAE493A3C8C582C8CCC583F4
:1044C500CCF0A3C8C582C8CCC583CCDFE9DEE780C4
:1044D5000D89828A83E493A3F608DFF9ECFAA9F043
:1044E500EDFB2289828A83ECFAE0A3C8C582C8CC99
:1044F500C583CCF0A3C8C582C8CCC583CCDFEADEB2
:10450500E880DB89828A83E493A3F208DFF980CC13
:1045150088F0EF60010E4E60C388F0ED2402B4040C
:104525000050B9F582EB2402B4040050AF232345B3
:06453500822390449573FF
:10453B00BB010689828A83E0225002E722BBFE027E
:09454B00E32289828A83E49322B1
:10455400BB010989828A83F8E028F022500327F7F7
:1045640022BBFE05F8E328F3228A838982F8E493C8
:024574002822FB
:10457600BB010689828A83F0225002F722BBFE0124
:02458600F3221E
:10458800EF8DF0A4A8F0CF8CF0A428CE8DF0A42E47
:02459800FE2201
:10459A00BC000BBE0029EF8DF084FFADF022E4CC05
:1045AA00F875F008EF2FFFEE33FEEC33FCEE9DECCE
:1045BA00984005FCEE9DFE0FD5F0E9E4CEFD22ED14
:1045CA00F8F5F0EE8420D21CFEADF075F008EF2F5E
:1045DA00FFED33FD4007985006D5F0F222C398FD4F
:0545EA000FD5F0EA22EC
:1045EF00A3F8E0C5F025F0F0E5821582700215837F
:0645FF00E0C838F0E822DC
:1046050075F008758200EF2FFFEE33FECD33CDCC6C
:1046150033CCC58233C5829BED9AEC99E5829840EF
:104625000CF582EE9BFEED9AFDEC99FC0FD5F0D6CC
:10463500E4CEFBE4CDFAE4CCF9A88222B800C1B9F6
:104645000059BA002DEC8BF084CFCECDFCE5F0CB34
:10465500F97818EF2FFFEE33FEED33FDEC33FCEB6D
:1046650033FB10D703994004EB99FB0FD8E5E4F928
:10467500FA227818EF2FFFEE33FEED33FDEC33FC15
:10468500C933C910D7059BE99A4007EC9BFCE99A09
:10469500F90FD8E0E4C9FAE4CCFB2275F010EF2F4E
:1046A500FFEE33FEED33FDCC33CCC833C810D7074E
:1046B5009BEC9AE899400AED9BFDEC9AFCE899F889
:0E46C5000FD5F0DAE4CDFBE4CCFAE4C8F9221C
:1046D300EB9FF5F0EA9E42F0E99D42F0E89C45F03D
:0146E30022B4
:1046E400E8600FECC313FCED13FDEE13FEEF13FFB4
:0346F400D8F122D8
:1046F700E8600FEFC333FFEE33FEED33FDEC33FC21
:03470700D8F122C4
:10470A007401FF3395E0FEFDFCA3A3A3E0CF2FF0D5
:10471A00E582158270021583E0CE3EF0E5821582AD
:10472A0070021583E0CD3DF0E58215827002158393
:05473A00E0CC3CF02280
:0C473F00ECF0A3EDF0A3EEF0A3EFF022ED
:10474B00A8828583F0D083D082124762124762120F
:10475B004762124762E473E493A3C583C5F0C58334
:10476B00C8C582C8F0A3C583C5F0C583C8C582C8B8
:01477B00221B
:0C477C00A42582F582E5F03583F5832248
:10478800D083D082F8E4937012740193700DA3A3C0
:1047980093F8740193F5828883E4737402936860D4
:0647A800EFA3A3A380DFD4
:0647AE008A838982E47396
:10480100E50D24A5F582E43405F583E0050D22903C
:1048110005A23007039005A5E475F0011247E102F6
:10482100453B2000E97F2ED2008018EF540F2490E1
:10483100D43440D4FF30040BEF24BFB41A0050032A
:104841002461FFE50E6002150E0511E511700205E8
:104851001030070E9005A2E475F0011247E1EF0256
:10486100457602679F7403D2078003E4C207F50D02
:104871009005A21247F8E4F50EF510F511E50E606A
:10488100077F2012484480F5750FFFC201C200C2A4
:1048910002C203C205C206C208124810FF700D30E1
:1048A10007057F00124855AF11AE1022B4255FC233
:1048B100D5C204124810FF24D0B40A00501A75F072
:1048C1000A780E30D50508B6FF0106C6A426F620E3
:1048D100D5047002D20380D924CFB41A00EF50045A
:1048E100C2E5D204024A56D20180C6D20080C0D2AB
:1048F1000280BCD2D580BAD20580B47F2012484450
:104901002002077401B50E0040F1124801FF124860
:104911004402487ED208D2068095124801FB124813
:1049210001FA124801F94A4B700679277A4B7BFF4D
:1049310020022EE50E602A7E008E827583001247CA
:10494100B460060EEE650F70F0C2D5EBC0E0EAC0B0
:10495100E0E9C0E0EE124A9DD0E0F9D0E0FAD0E003
:10496100FB12453BFF60AAEBC0E0EAC0E0E9C0E012
:10497100124844D0E02401F9D0E03400FAD0E0FB41
:10498100E50F0460DCD50FD980877BFF7A4A7999DE
:10499100D202809C791080027908C206C208800880
:1049A100D2D5790A8004790AC2D5E50F047002F5DF
:1049B1000FE4FAFDFEFF124801FC7B0820011312EF
:1049C1004801FD7B1030000A124801FE124801FF28
:1049D1007B20EC3382D592D55013C3E43000069F7F
:1049E100FFE49EFEE42001039DFDE49CFCE4CBF882
:1049F100C201EC700CCFCECDCCE824F8F870F38076
:104A010017C3EF33FFEE33FEED33FDEC33FCEB3335
:104A1100FB994002FB0FD8E9EB300105F8D0E0C467
:104A210048B201C0E00AEC4D4E4F78207B0070C2C5
:104A3100EAB50F0040BCC0E0124A9FD0F0D0E020A0
:104A41000104C4C0E0C4B201C0F012482DD0F0D5B9
:104A5100F0EB02487E124788491B5349955848ECB0
:104A61004C48E84249994F49A14449A14949014368
:084A710049A755498B46498B0A
:104A790045498B474B475048F02D48F42E49172B91
:104A890048F8234915204B302A48B0480000490FFF
:104A99003F3F3F00790AA2D5200314300509B91018
:104AA900020404B9080104A2D52006025001042019
:104AB90002689202B50E005034C0E07F203003191D
:104AC9007F30A20272067205500F124AF6C202C264
:104AD90006C205C2087F30800F300503E9C0E01225
:104AE9004844300503D0E0F9D0E0B50ECC300517C5
:104AF9007F30B9100C1248447F583004077F788002
:104B090003B908031248443002057F2D0248447F47
:104B1900202008F87F2B2006F322920280CF286EEE
:104B2900756C6C2900D2011248013001F8C2017874
:104B39000E30D50108F60248B02D504349581248A5
:104B4900012403B405004001E4904B429312483517
:0D4B5900743A124835D203750E04024995D6
:1047B400BB010CE58229F582E5833AF583E02250BA
:1047C40006E92582F8E622BBFE06E92582F8E22204
:0D47D400E58229F582E5833AF583E493221E
:1047E100F8E0FBA3A3E0F925F0F0E5821582700261
:0747F1001583E0FA38F02205
:0947F800EBF0A3EAF0A3E9F022C2
:10679F00EFB40A07740D1267AA740A309811A899FA
:1067AF00B8130CC2983098FDA899C298B811F6305A
:0767BF0099FDC299F5992232
:00000001FF
